******************************************************************************
                  TI ARM Linker PC v20.2.5                     
******************************************************************************
>> Linked Wed Oct 18 10:29:26 2023

OUTPUT FILE NAME:   <DMA2.out>
ENTRY POINT SYMBOL: "_c_int00"  address: 000053d8


MEMORY CONFIGURATION

         name            origin    length      used     unused   attr    fill
----------------------  --------  ---------  --------  --------  ----  --------
  VECTORS               00000000   00000020  00000020  00000000     X
  FLASH0                00000020   001fffe0  000057b8  001fa828  R  X
  FLASH1                00200000   00200000  00000000  00200000  R  X
  STACKS                08000000   00001500  00000000  00001500  RW  
  RAM                   08001500   0007eb00  000000b4  0007ea4c  RW  


SEGMENT ALLOCATION MAP

run origin  load origin   length   init length attrs members
----------  ----------- ---------- ----------- ----- -------
00000000    00000000    000055c4   000055c4    r-x
  00000000    00000000    00000020   00000020    r-x .intvecs
  00000020    00000020    000055a4   000055a4    r-x .text
000055e0    000055e0    00000214   00000214    r--
  000055e0    000055e0    00000200   00000200    r-- .const
  000057e0    000057e0    00000014   00000014    r-- .cinit
08001500    08001500    000000b4   00000000    rw-
  08001500    08001500    000000b4   00000000    rw- .bss


SECTION ALLOCATION MAP

 output                                  attributes/
section   page    origin      length       input sections
--------  ----  ----------  ----------   ----------------
.intvecs   0    00000000    00000020     
                  00000000    00000020     HL_sys_intvecs.obj (.intvecs)

.text      0    00000020    000055a4     
                  00000020    00000ff4     HL_sci.obj (.text)
                  00001014    000009cc     HL_pinmux.obj (.text)
                  000019e0    00000998     HL_system.obj (.text)
                  00002378    00000938     HL_sys_vim.obj (.text)
                  00002cb0    00000920     HL_sys_dma.obj (.text)
                  000035d0    0000078c     HL_esm.obj (.text)
                  00003d5c    00000664     HL_errata_SSWF021_45.obj (.text)
                  000043c0    000003c4     HL_sys_core.obj (.text)
                  00004784    0000036c     HL_sys_mpu.obj (.text)
                  00004af0    0000033c     HL_sys_vim.obj (.text:retain)
                  00004e2c    00000180     rtsv7R4_A_be_v3D16_eabi.lib : memcpy32.asm.obj (.text)
                  00004fac    00000178     HL_sys_main.obj (.text)
                  00005124    00000178     HL_esm.obj (.text:retain)
                  0000529c    0000013c     rtsv7R4_A_be_v3D16_eabi.lib : s_floor.c.obj (.text:floor)
                  000053d8    000000d8     HL_sys_startup.obj (.text:retain)
                  000054b0    00000074     HL_notification.obj (.text)
                  00005524    00000068     rtsv7R4_A_be_v3D16_eabi.lib : autoinit.c.obj (.text:__TI_auto_init_nobinit_nopinit:__TI_auto_init_nobinit_nopinit)
                  0000558c    00000028                                 : copy_zero_init.c.obj (.text:decompress:ZI:__TI_zero_init_nomemset:__TI_zero_init_nomemset)
                  000055b4    00000008                                 : exit.c.obj (.text:abort:abort)
                  000055bc    00000004     HL_sys_startup.obj (.text)
                  000055c0    00000004     HL_sys_phantom.obj (.text:retain)

.const     0    000055e0    00000200     
                  000055e0    00000200     HL_sys_vim.obj (.const:s_vim_init)

.cinit     0    000057e0    00000014     
                  000057e0    00000008     (.cinit..bss.load) [load image, compression = zero_init]
                  000057e8    00000004     (__TI_handler_table)
                  000057ec    00000008     (__TI_cinit_table)

.bss       0    08001500    000000b4     UNINITIALIZED
                  08001500    00000064     (.common:TX_DATA)
                  08001564    00000050     HL_sci.obj (.bss:g_sciTransfer_t)

__llvm_prf_cnts 
*          0    08001500    00000000     UNINITIALIZED

MODULE SUMMARY

       Module                     code    ro data   rw data
       ------                     ----    -------   -------
    .\source\
       HL_sci.obj                 4084    0         80     
       HL_sys_vim.obj             3188    512       0      
       HL_pinmux.obj              2508    0         0      
       HL_system.obj              2456    0         0      
       HL_sys_dma.obj             2336    0         0      
       HL_esm.obj                 2308    0         0      
       HL_errata_SSWF021_45.obj   1636    0         0      
       HL_sys_core.obj            964     0         0      
       HL_sys_mpu.obj             876     0         0      
       HL_sys_main.obj            376     0         100    
       HL_sys_startup.obj         220     0         0      
       HL_notification.obj        116     0         0      
       HL_sys_intvecs.obj         32      0         0      
       HL_sys_phantom.obj         4       0         0      
    +--+--------------------------+-------+---------+---------+
       Total:                     21104   512       180    
                                                           
    C:\ti\ccs1120\ccs\tools\compiler\ti-cgt-arm_20.2.5.LTS\lib\rtsv7R4_A_be_v3D16_eabi.lib
       memcpy32.asm.obj           384     0         0      
       s_floor.c.obj              316     0         0      
       autoinit.c.obj             104     0         0      
       copy_zero_init.c.obj       40      0         0      
       exit.c.obj                 8       0         0      
    +--+--------------------------+-------+---------+---------+
       Total:                     852     0         0      
                                                           
       Linker Generated:          0       20        0      
    +--+--------------------------+-------+---------+---------+
       Grand Total:               21956   532       180    


LINKER GENERATED COPY TABLES

__TI_cinit_table @ 000057ec records: 1, size/record: 8, table size: 8
	.bss: load addr=000057e0, load size=00000008 bytes, run addr=08001500, run size=000000b4 bytes, compression=zero_init


LINKER GENERATED HANDLER TABLE

__TI_handler_table @ 000057e8 records: 1, size/record: 4, table size: 4
	index: 0, handler: __TI_zero_init


GLOBAL SYMBOLS: SORTED ALPHABETICALLY BY Name 

address   name                                
-------   ----                                
000055b4  C$$EXIT                             
UNDEFED   SHT$$INIT_ARRAY$$Base               
UNDEFED   SHT$$INIT_ARRAY$$Limit              
08001500  TX_DATA                             
000057ec  __TI_CINIT_Base                     
000057f4  __TI_CINIT_Limit                    
000057e8  __TI_Handler_Table_Base             
000057ec  __TI_Handler_Table_Limit            
0000477c  __TI_PINIT_Base                     
00004780  __TI_PINIT_Limit                    
00005524  __TI_auto_init_nobinit_nopinit      
ffffffff  __TI_pprof_out_hndl                 
ffffffff  __TI_prof_data_size                 
ffffffff  __TI_prof_data_start                
00000000  __TI_static_base__                  
0000558c  __TI_zero_init_nomemset             
00004e2c  __aeabi_memcpy                      
00004e2c  __aeabi_memcpy4                     
00004e2c  __aeabi_memcpy8                     
ffffffff  __binit__                           
ffffffff  __c_args__                          
08001500  __start___llvm_prf_cnts             
08001500  __stop___llvm_prf_cnts              
000053d8  _c_int00                            
00004730  _cacheDisable_                      
000046ec  _cacheEnable_                       
000046cc  _checkMemInitOn_                    
000045d8  _coreClearAuxiliaryDataFault_       
000045ec  _coreClearAuxiliaryInstructionFault_
000045b0  _coreClearDataFaultAddress_         
00004588  _coreClearDataFault_                
000045c4  _coreClearInstructionFaultAddress_  
0000459c  _coreClearInstructionFault_         
00004560  _coreDisableEventBusExport_         
00004550  _coreEnableEventBusExport_          
00004570  _coreEnableIrqVicOffset_            
00004538  _coreEnableVfp_                     
000045d0  _coreGetAuxiliaryDataFault_         
000045e4  _coreGetAuxiliaryInstructionFault_  
000045a8  _coreGetDataFaultAddress_           
00004580  _coreGetDataFault_                  
000045bc  _coreGetInstructionFaultAddress_    
00004594  _coreGetInstructionFault_           
000043c0  _coreInitRegisters_                 
000044cc  _coreInitStackPointer_              
00004754  _dCacheInvalidate_                  
000045f8  _disable_IRQ_interrupt_             
00004600  _enable_IRQ_interrupt_              
00004608  _enable_interrupt_                  
00003d5c  _errata_SSWF021_45_both_plls        
00003f50  _errata_SSWF021_45_pll1             
000040c8  _errata_SSWF021_45_pll2             
00004610  _esmCcmErrorsClear_                 
00004518  _getCPSRValue_                      
00004520  _gotoCPUIdle_                       
00004768  _iCacheInvalidate_                  
00004698  _memInit_                           
00004a98  _mpuAreRegionsSeparate_             
00004a7c  _mpuDisableBackgroundRegion_        
00004a54  _mpuDisable_                        
00004a6c  _mpuEnableBackgroundRegion_         
00004a3c  _mpuEnable_                         
00004a8c  _mpuGetNumberOfRegions_             
00004abc  _mpuGetRegionBaseAddress_           
00004adc  _mpuGetRegionPermission_            
00004ad0  _mpuGetRegionType_                  
00004aac  _mpuGetRegion_                      
00004784  _mpuInit_                           
00004ab4  _mpuSetRegionBaseAddress_           
00004ae8  _mpuSetRegionSizeRegister_          
00004ac4  _mpuSetRegionTypeAndPermission_     
00004aa4  _mpuSetRegion_                      
UNDEFED   _system_post_cinit                  
000055b4  abort                               
ffffffff  binit                               
000022d0  customTrimLPO                       
00003158  dmaDefineRegion                     
00002cd0  dmaDisable                          
00003340  dmaDisableECC                       
000030b8  dmaDisableInterrupt                 
000032bc  dmaDisableRegion                    
00002cb0  dmaEnable                           
00003330  dmaEnableECC                        
00002f64  dmaEnableInterrupt                  
000031d4  dmaEnableRegion                     
00003428  dmaGetInterruptStatus               
00003350  dmaGetReq                           
000054e8  dmaGroupANotification               
000033f4  dmaIsBusy                           
000033a8  dmaIsChannelActive                  
00002e94  dmaReqAssign                        
00002e48  dmaSetChEnable                      
00002cf0  dmaSetCtrlPacket                    
00002f18  dmaSetPriority                      
00005510  epcCAMFullNotification              
00005514  epcFIFOFullNotification             
000037e0  esmActivateNormalOperation          
0000392c  esmClearStatus                      
00003990  esmClearStatusBuffer                
0000396c  esmClearStatusUpper                 
0000378c  esmDisableError                     
000037b4  esmDisableErrorUpper                
00003834  esmDisableInterrupt                 
0000385c  esmDisableInterruptUpper            
00003748  esmEnableError                      
00003770  esmEnableErrorUpper                 
000037f0  esmEnableInterrupt                  
00003818  esmEnableInterruptUpper             
00003ac0  esmEnterSelfTest                    
0000372c  esmError                            
00003b98  esmGetConfigValue                   
000039cc  esmGetStatus                        
00003a98  esmGetStatusBuffer                  
00003a50  esmGetStatusUpper                   
000054b0  esmGroup1Notification               
000054c4  esmGroup2Notification               
000054d8  esmGroup3Notification               
00005124  esmHighInterrupt                    
000035d0  esmInit                             
00003b48  esmSelfTestStatus                   
000039ac  esmSetCounterPreloadValue           
00003878  esmSetInterruptLevel                
000038ec  esmSetInterruptLevelUpper           
000037d0  esmTriggerErrorPinReset             
0000529c  floor                               
0000529c  floorl                              
00001d78  getResetSource                      
000055bc  handlePLLLockFail                   
00004fac  main                                
00001ba8  mapClocks                           
00004e2c  memcpy                              
00001014  muxInit                             
00001af4  periphInit                          
000055c0  phantomInterrupt                    
00000000  resetEntry                          
00000994  sci1GetConfigValue                  
00000aec  sci2GetConfigValue                  
00000c44  sci3GetConfigValue                  
00000d9c  sci4GetConfigValue                  
00000808  sciDisableLoopback                  
000008bc  sciDisableNotification              
000007d4  sciEnableLoopback                   
00000824  sciEnableNotification               
00000954  sciEnterResetState                  
00000974  sciExitResetState                   
00000020  sciInit                             
0000064c  sciIsIdleDetected                   
00000630  sciIsRxReady                        
00000480  sciIsTxReady                        
000054fc  sciNotification                     
000006c4  sciReceive                          
00000698  sciReceiveByte                      
00000668  sciRxError                          
000004cc  sciSend                             
0000049c  sciSendByte                         
000003e4  sciSetBaudrate                      
000003c4  sciSetFunctional                    
00001ab4  setupFlash                          
000019e0  setupPLL                            
00001ea0  systemGetConfigValue                
00001cd4  systemInit                          
00001d48  systemPowerDown                     
00001a40  trimLPO                             
0000244c  vimChannelMap                       
000026b8  vimDisableInterrupt                 
00004af0  vimECCErrorHandler                  
000024f0  vimEnableInterrupt                  
00002764  vimGetConfigValue                   
00002378  vimInit                             


GLOBAL SYMBOLS: SORTED BY Symbol Address 

address   name                                
-------   ----                                
00000000  __TI_static_base__                  
00000000  resetEntry                          
00000020  sciInit                             
000003c4  sciSetFunctional                    
000003e4  sciSetBaudrate                      
00000480  sciIsTxReady                        
0000049c  sciSendByte                         
000004cc  sciSend                             
00000630  sciIsRxReady                        
0000064c  sciIsIdleDetected                   
00000668  sciRxError                          
00000698  sciReceiveByte                      
000006c4  sciReceive                          
000007d4  sciEnableLoopback                   
00000808  sciDisableLoopback                  
00000824  sciEnableNotification               
000008bc  sciDisableNotification              
00000954  sciEnterResetState                  
00000974  sciExitResetState                   
00000994  sci1GetConfigValue                  
00000aec  sci2GetConfigValue                  
00000c44  sci3GetConfigValue                  
00000d9c  sci4GetConfigValue                  
00001014  muxInit                             
000019e0  setupPLL                            
00001a40  trimLPO                             
00001ab4  setupFlash                          
00001af4  periphInit                          
00001ba8  mapClocks                           
00001cd4  systemInit                          
00001d48  systemPowerDown                     
00001d78  getResetSource                      
00001ea0  systemGetConfigValue                
000022d0  customTrimLPO                       
00002378  vimInit                             
0000244c  vimChannelMap                       
000024f0  vimEnableInterrupt                  
000026b8  vimDisableInterrupt                 
00002764  vimGetConfigValue                   
00002cb0  dmaEnable                           
00002cd0  dmaDisable                          
00002cf0  dmaSetCtrlPacket                    
00002e48  dmaSetChEnable                      
00002e94  dmaReqAssign                        
00002f18  dmaSetPriority                      
00002f64  dmaEnableInterrupt                  
000030b8  dmaDisableInterrupt                 
00003158  dmaDefineRegion                     
000031d4  dmaEnableRegion                     
000032bc  dmaDisableRegion                    
00003330  dmaEnableECC                        
00003340  dmaDisableECC                       
00003350  dmaGetReq                           
000033a8  dmaIsChannelActive                  
000033f4  dmaIsBusy                           
00003428  dmaGetInterruptStatus               
000035d0  esmInit                             
0000372c  esmError                            
00003748  esmEnableError                      
00003770  esmEnableErrorUpper                 
0000378c  esmDisableError                     
000037b4  esmDisableErrorUpper                
000037d0  esmTriggerErrorPinReset             
000037e0  esmActivateNormalOperation          
000037f0  esmEnableInterrupt                  
00003818  esmEnableInterruptUpper             
00003834  esmDisableInterrupt                 
0000385c  esmDisableInterruptUpper            
00003878  esmSetInterruptLevel                
000038ec  esmSetInterruptLevelUpper           
0000392c  esmClearStatus                      
0000396c  esmClearStatusUpper                 
00003990  esmClearStatusBuffer                
000039ac  esmSetCounterPreloadValue           
000039cc  esmGetStatus                        
00003a50  esmGetStatusUpper                   
00003a98  esmGetStatusBuffer                  
00003ac0  esmEnterSelfTest                    
00003b48  esmSelfTestStatus                   
00003b98  esmGetConfigValue                   
00003d5c  _errata_SSWF021_45_both_plls        
00003f50  _errata_SSWF021_45_pll1             
000040c8  _errata_SSWF021_45_pll2             
000043c0  _coreInitRegisters_                 
000044cc  _coreInitStackPointer_              
00004518  _getCPSRValue_                      
00004520  _gotoCPUIdle_                       
00004538  _coreEnableVfp_                     
00004550  _coreEnableEventBusExport_          
00004560  _coreDisableEventBusExport_         
00004570  _coreEnableIrqVicOffset_            
00004580  _coreGetDataFault_                  
00004588  _coreClearDataFault_                
00004594  _coreGetInstructionFault_           
0000459c  _coreClearInstructionFault_         
000045a8  _coreGetDataFaultAddress_           
000045b0  _coreClearDataFaultAddress_         
000045bc  _coreGetInstructionFaultAddress_    
000045c4  _coreClearInstructionFaultAddress_  
000045d0  _coreGetAuxiliaryDataFault_         
000045d8  _coreClearAuxiliaryDataFault_       
000045e4  _coreGetAuxiliaryInstructionFault_  
000045ec  _coreClearAuxiliaryInstructionFault_
000045f8  _disable_IRQ_interrupt_             
00004600  _enable_IRQ_interrupt_              
00004608  _enable_interrupt_                  
00004610  _esmCcmErrorsClear_                 
00004698  _memInit_                           
000046cc  _checkMemInitOn_                    
000046ec  _cacheEnable_                       
00004730  _cacheDisable_                      
00004754  _dCacheInvalidate_                  
00004768  _iCacheInvalidate_                  
0000477c  __TI_PINIT_Base                     
00004780  __TI_PINIT_Limit                    
00004784  _mpuInit_                           
00004a3c  _mpuEnable_                         
00004a54  _mpuDisable_                        
00004a6c  _mpuEnableBackgroundRegion_         
00004a7c  _mpuDisableBackgroundRegion_        
00004a8c  _mpuGetNumberOfRegions_             
00004a98  _mpuAreRegionsSeparate_             
00004aa4  _mpuSetRegion_                      
00004aac  _mpuGetRegion_                      
00004ab4  _mpuSetRegionBaseAddress_           
00004abc  _mpuGetRegionBaseAddress_           
00004ac4  _mpuSetRegionTypeAndPermission_     
00004ad0  _mpuGetRegionType_                  
00004adc  _mpuGetRegionPermission_            
00004ae8  _mpuSetRegionSizeRegister_          
00004af0  vimECCErrorHandler                  
00004e2c  __aeabi_memcpy                      
00004e2c  __aeabi_memcpy4                     
00004e2c  __aeabi_memcpy8                     
00004e2c  memcpy                              
00004fac  main                                
00005124  esmHighInterrupt                    
0000529c  floor                               
0000529c  floorl                              
000053d8  _c_int00                            
000054b0  esmGroup1Notification               
000054c4  esmGroup2Notification               
000054d8  esmGroup3Notification               
000054e8  dmaGroupANotification               
000054fc  sciNotification                     
00005510  epcCAMFullNotification              
00005514  epcFIFOFullNotification             
00005524  __TI_auto_init_nobinit_nopinit      
0000558c  __TI_zero_init_nomemset             
000055b4  C$$EXIT                             
000055b4  abort                               
000055bc  handlePLLLockFail                   
000055c0  phantomInterrupt                    
000057e8  __TI_Handler_Table_Base             
000057ec  __TI_CINIT_Base                     
000057ec  __TI_Handler_Table_Limit            
000057f4  __TI_CINIT_Limit                    
08001500  TX_DATA                             
08001500  __start___llvm_prf_cnts             
08001500  __stop___llvm_prf_cnts              
ffffffff  __TI_pprof_out_hndl                 
ffffffff  __TI_prof_data_size                 
ffffffff  __TI_prof_data_start                
ffffffff  __binit__                           
ffffffff  __c_args__                          
ffffffff  binit                               
UNDEFED   SHT$$INIT_ARRAY$$Base               
UNDEFED   SHT$$INIT_ARRAY$$Limit              
UNDEFED   _system_post_cinit                  

[169 symbols]
